:040000008A11302F02
:100E020064008001840A0406031900340406022FD8
:100E12007E088A007F08820009278A118000840ADE
:100E220004087D0603190034FF0A0319FE0A0D2F78
:100E3200282FF930F2006400F20B1C2F202F6400DF
:100E4200FF30F0070318F10AFF30F107282F71086D
:100E52007004031D2D2F2E2F1A2F2F2F0800FB0198
:100E6200FC01FD0183134030840050308A110127B8
:100E72008A114030FD000730FE004830FF0020306C
:100E820084008A110D278A1183018A119F2F303421
:100E9200313432343334343435343634373438340C
:100EA2003934413442344334443445344634EE34E4
:100EB200ED34EB34E734DE34DD34DB34D734BE34A6
:100EC200BD34BB34B7347E347D347B347734003068
:100ED200FA000030F9000030F8000030F700872FE8
:100EE200E830F0000330F1008A1119278A1101302D
:100EF200F707003003180130F807003003180130FB
:100F0200F907003003180130FA07872F7A08803A70
:100F1200FF007608803A7F02031D992F7508790237
:100F2200031D992F74087802031D992F7308770205
:100F3200031C9C2F9D2F712F9E2F080083120313D9
:100F420098130730831603139C009D019B01003008
:100F520083120313DB000030DA000030D9000230C4
:100F6200D8000030D3000030D2000030D10002306F
:100F7200D0000030D7000030D6000030D50002305B
:100F8200D400831603138501FF30860083120313F6
:100F92008501831603138113CE2F831205145B0878
:100FA200F6005A08F5005908F4005808F3008A11AF
:100FB20068278A1183120313051085145308F6005B
:100FC2005208F5005108F4005008F3008A1168270E
:100FD2008A1183120313851005155708F600560867
:100FE200F5005508F4005408F3008A1168278A11A5
:0E0FF200831203130511CE2FCE2F8A11002873
:00000001FF
